:030000000219FDE5
:03000B000200A848
:03002B0002019738
:03005B000203415C
:030073000203275E
:1000800002030406080C10182030406080040608A3
:100090000C10182030406080A0C000070F1F3F05E3
:1000A000050D050305030302C2AF306308C2638573
:1000B0007C8AD2AF32C0D0C0E0206227E525600242
:1000C000E473E525F4C3334009758A00D263F57CF7
:1000D00001D4F58A758B00758D00D262D0E0D0D046
:1000E000D2AF32C3E526334009758A00D263F57C6E
:1000F00001F4F58AC262E526F4603B3068032072A1
:1001000013758B00758D00D0E0D0D0C292C296C21C
:1001100094D2AF32C292C296C294206E0C2066096D
:10012000740ED5E0FDE57E4290758B00758D00D094
:10013000E0D0D0D2AF32758A00D263757C00C28D18
:10014000D262212901C2306805206602D29201C222
:10015000306805206602D29401C23068052066022C
:10016000D29601C2C29330680A2066077410D5E0A7
:10017000FDD29201C2C29530680A2066077410D57C
:10018000E0FDD29401C2C29730680A20660774105D
:10019000D5E0FDD29601C2C2AFC2AD53E6EFC0D0EA
:1001A000C0E0D2D3D2AFE57D6009E57A6005757A0B
:1001B0000041D4757A01C2CEE52A60072074491542
:1001C0002A41087800790020742EE580307E01F401
:1001D00030E50278FF53DACF207E0343DA20307E09
:1001E0000343DA10C2D8C271E580307E01F430E5F5
:1001F0000279FFC3E89970CB306103752A18207427
:1002000003752A18885FD27020740DE52B600415E1
:100210002B411843DA01C2D8207002417AA85F202E
:100220006102C270207431C3E894F0400374F0F8A6
:10023000E8C4540F28F87984B703024158C313C3A4
:10024000138721200802C313200A06C3C898F84167
:100250005828F8500374FFF8C3E895685003E56820
:10026000F88822E52D54066011E533C313C3132427
:10027000062522F52250037522FF852224A824C3D7
:10028000E52495644002A8648825E569700241BEB2
:10029000C3E8AA699A5003E8FAE4F9EAC333FBE534
:1002A0006BF45B29400D256AF8E56A6002156A4027
:1002B0000B41BE0AC3E56A9A5002056A78FF882698
:1002C000C26EC3E52694F84002D26EC3E525944081
:1002D0004002D26420CF0AD0E0D0D043E610D2ADA5
:1002E00032C2CF053AE57D6009E57B6005757B008C
:1002F000611D757B017801E52A6005307402152ABD
:10030000C3E55F94014005756200611D756300756A
:100310006C00E5622401F56250037562FFD0E0D005
:10032000D043E610D2AD32C2AFC0D053E67FC26038
:10033000759100855694855795759104D0D0D2AFAC
:1003400032C2AF53E6EFC2ADC0D0C0E0C0F0D2D3EE
:10035000D2AFA8FBA9FCE57D6007C3E913F9E81358
:10036000F8C2D830710261B353DACF207E0343DA8A
:1003700010307E0343DA20D271E580307E01F42014
:10038000E502618A88278928A1DA53DACF207E0323
:1003900043DA20307E0343DA10C2D8C271307402CF
:1003A000A1C67800E580307E01F430E502A1C68860
:1003B0005FA1AE53DACF207E0343DA20307E0343C1
:1003C000DA10C271206102818C53DACF207E0343A0
:1003D000DA10307E0343DA20C2D8D271885A895BA2
:1003E000C3E89558F8E99559F97B007E087A00C36F
:1003F000E8948CE994005005755E00817E88217830
:10040000A2E6A8216055C3E894C8E994005008E426
:10041000D2E4FB7A0A8159C3E89468E99401500850
:10042000E4D2E3FB7A0F8159C3E894D0E9940250F7
:1004300008E4D2E2FB7A1E8159C3E894A0E994054E
:100440005008E4D2E1FB7A3C8159C3E89498E994DE
:10045000085008E4D2E0FB7A787E00C3E8955CFCA3
:10046000E9955DFD30E70AECF42401FCEDF434007D
:0E047000FD755E00C3EC9AED9E5003755E01B3
:10047E00885C895D855A58855B597802A1AEC3E8C0
:10048E009527F8E99528F9307C02A192307B02A1DC
:10049E0092307A02A18B20750281AFE9FDE8FC81D2
:1004AE00CEE9C313F9E813F8307902A18BE9C3132F
:1004BE00F9E813F8307802A18BE9C313FDE813FCB9
:1004CE00206126C3EC941CED9402400281E5ED7090
:1004DE0018C3EC94C850120529C3E529940A50029A
:1004EE00A1C6755F00D270A1C6E5296002152978F4
:1004FE0088E6F97400207F087896B90302789EE6A4
:10050E0024FAFEE43400FFC3EC9EFCED9FFD92083E
:10051E00B90310A2085007207609D276A1313076A1
:10052E0002C276A2085016B9030DECF42401FCEDBC
:10053E00F43400FD02054B78007900A192B9031541
:10054E00EC33FCED33FDC3EC940AFCED9400FD504E
:10055E00047C007D00C3EC94FFED9400400678FF10
:10056E007900A192EC8575F0A4C5F0A2F733F87965
:10057E000040030205AE78FF79000205AEE9C31311
:10058E00F9E813F8307C0EE9600278FFC3E81338FF
:10059E00F8E43400F9C3E894FFE99400400278FFD0
:1005AE00885FD270206102A1C6741FF4552F4BF5DF
:1005BE002FC274EB7002D274752A18307403752A28
:1005CE000A306102A1DA20740353DAFE2074037537
:1005DE002B06D0F0D0E0D0D0D2AD43E61032790168
:1005EE0002060A790302060A790A02060A791E022F
:1005FE00060A796402060A79C802060A7817E4D553
:10060E00E0FDD8FAD9F6227A147B780206317A10F8
:10061E007B8C0206317A0D7BB40206317A0B7BC8D5
:10062E000206317902B27DE4C295D5E0FDD294D5B1
:10063E00E0FDC294D5E0FDD295D5E0FDD292E576EF
:10064E00D5E0FDC2927496D5E0FDD9D9EAF8D5E091
:10065E00FDD8FBDBCEC29522C37C007D0075F00079
:10066E0005F0EA33FAEB33FB50F6EB13FBEA13FA21
:10067E00C3E9FFE8FEE89AF8E99BF95004EFF9EEBA
:10068E00F8B3EC33FCED33FDD5F0DFEDF9ECF822E9
:10069E00E889F08A20D2D4F8A9F07B0030F70B7BE2
:1006AE00FFF42401F8E9F43400F9E88520F0A4AD54
:1006BE00F0F8E98520F0A4AFF0FEED2EF974003FBE
:1006CE00FA7C04C3EA13FAE913F9E813F8DCF48BA5
:1006DE00F030F70AE8F42401F8E9F43400F9E88977
:1006EE00F0C2D4F8A9F02222C3E54113F9E5401374
:1006FE00F8C3E54598F8E54699F9500CC3E894809F
:10070E00E994FF401602072DC3E8947FE994005048
:10071E000302072D787F790002072D788079FF88F4
:10072E004A894B22E54A2547F8E54B3548F9854B72
:10073E0020E4300701F43549FA30E709C3EA94F0B2
:10074E00401502076BC3EA940F500302076B78FF44
:10075E0079FF7A0F02076B780079007AF0C3E524EF
:10076E009564500AC374019524500B020789E54B1A
:10077E0020E70E020789E54B30E706884789488A4D
:10078E00492278A4E6FAC3E54A33F8E54B33F9D1AA
:10079E009EE930E70BC3E89480E994FF4013E1C370
:1007AE00C3E8947FE994005002E1C3787F7900E1B9
:1007BE00C3788079FFE820E715C3E52398F8400950
:1007CE00C3E8940140030207EA78010207EAE8F45D
:1007DE0024012523F840030207EA78FF884C22788B
:1007EE00A5E6FAA848A949D19EE930E70CC3E894DA
:1007FE0001E994FF401602081EC3E894FFE9940035
:10080E00500302081E78FF790002081E780179FF56
:10081E00E920E715C3E54C98F84009C3E894014078
:10082E00030208457801020845E8F42401254CF836
:10083E00400302084578FF88242278FFC2642069AD
:10084E003D206A12D264C3E541940A4009C3E525EE
:10085E0094405002C26479A1E76023E541601F74A1
:0F086E00FF8541F0848539F0306A0375F005A4E9
:10087D00F8C5F0600278FFC3E895675002A8678855
:10088D006622C3E54094C8E5419400E56650031423
:10089D0001A0046002F566220208A82275E89022E4
:1008AD007883E6FFE5E820ECF7A8BDA9BE0573C384
:1008BD00E57394084052757300E9FA79A0E7604436
:1008CD00EA7007E574601B0208E3C3E895746010D5
:1008DD00E5745006600C140208EF0460F90208EF8D
:1008ED00E574F574C39472401B7564C0C3940440E1
:1008FD0013756480C39404400B756440C394044025
:10090D000375640075BB0822E564F460020564E5B7
:10091D0073B4070375BB1022743279A687F0A4C592
:10092D00F0A2F733F8C3E895644002A864882288E2
:10093D0024882588268867227540007541F022C2DB
:10094D00AF75C820A8CCA9CDAA3A30CF010A75C879
:10095D0024D2AFC3EA13FAE913F9E813F8AB3BACB1
:10096D003C883B893CC3E89BF8E99C20690A547F8D
:10097D00F9306702416F21CCAD3D8A3DF9EA9D54B6
:10098D007FFA600478FF79FFAE3EAF3F8B3E8C3F20
:10099D00C3EC9FFCC3E99CF542A83BA93CC3E89E70
:1009AD00F8E99FF9C3E54113FBE54013FAE82AF591
:1009BD0040E93BF54150067540FF7541FF4116AAD0
:1009CD0040AB41AC40AD417E047F02C3EB9404408B
:1009DD00021E1FC3EB940840021E1FC3ED13FDEC56
:1009ED0013FCDEF7C3EA9CFAEB9DFBEF6009C3E94C
:1009FD0013F9E813F8DFF7EA28FAEB39FB8A408B95
:100A0D004150067BFF8B408B41C3EB94025002D2C9
:100A1D00673069047F0341417892E6FFC3E537945F
:100A2D008240110FC3E53794A040010FC3EF940628
:100A3D0040027F057E03E541C4540FF9E541C454DE
:100A4D00F0F8E540C4540F28F8C3E89EFAE9940085
:100A5D00FB4009C3EA9402EB940050047A02E4FBD4
:100A6D0041BBAA40AB41EBC4FEEAC4540F4EFCC3DC
:100A7D00EA9CFAEB9400FBC3E813C313F8EA28FAD7
:100A8D00EB3400FB8A408B41C3EB94024002C267FA
:100A9D007803EBC4FE7B00EAC4540F4EFAC3EA9808
:100AAD00FA4005C3940250027A027892E6FF306054
:100ABD000241BB855256855357D26043E680C3E44D
:100ACD009AF8E49BF9C3E833F8E933F9306702612A
:100ADD005CE8FAE9FBD3E913FDE813FC885289536E
:100AED00C3EF94036038EF20E00DE82CF8E93DF9F1
:100AFD00ECFAEDFB020B17E828F8E939F9C3E82405
:100B0D0002F8E93400F97AFE7BFFC3EF9403400E3F
:100B1D008A548B55884E894F8C508D5161908854D5
:100B2D0089558A4E8B4F8C508D51306920C3E533DA
:100B3D0094034019E542A2E713F8E555F424013872
:100B4D00400B20E7087554FFF42401F5556190E83A
:100B5D00FAD3E813FC8852C3EF94036020EF20E032
:100B6D0007E82CF8ECFA617CE8282402F87AFEC339
:100B7D00EF940340088A54884E8C50619088548AB3
:100B8D004E8C50E56BC3335002646BF56B306002D5
:100B9D00619A753404D26043E680E52D5406601FDA
:100BAD00A840A941C2AF53E67F759100C3E498F503
:100BBD0094E499F595759104D26043E680D2AF2205
:100BCD00D265754400752000306B03752040020B13
:100BDD00ECD265754400752040306B03752000D252
:100BED00AF7801206722E52D54066002C265C3E58A
:100BFD00419405401378029405400878039405400C
:100C0D00027806306902780A206019E544601530D3
:100C1D00690AC3E53394034003D53406D2AFD26CD1
:100C2D0081CF71A2D2AF0000C2AF20672AE541C3C8
:100C3D00FB940F40027B0FEB240530730123306AC8
:100C4D0002742820620123F93069027982E58D133F
:100C5D00E58B13C39940B10544E59BF45440B52091
:0E0C6D000281B930690A08C3E8940A40010800
:100C7B00811520650261ECC26553E67F75910030EA
:100C8B0067107594007595FC759104D26043E680EE
:100C9B0061ECAE40AF41C3EE33FEEF33FF50047E49
:100CAB00FF7FFFC3E49EF594E49FF5958193C3E525
:100CBB00339402500261EC30650261ECD80281CDB5
:100CCB008115C26C53E67F759100855494855595BB
:100CDB00759104854E56854F57D26043E680D2AF4F
:100CEB00E52D54066008206A020533020D09306CAD
:100CFB000D206B0A206507158115810215A7227837
:100D0B00003064053065027801E53775F007A4F90A
:100D1B00E5F028F5F0E9A2F013A2F113A2F213F516
:100D2B0037C394785003753778C3E5379538400847
:100D3B00D266C292C296C294306002A143855056CD
:100D4B00855157D26043E68022207D11C2AF754397
:100D5B0002C295D293D2AF759F40020F23C2AF75DB
:100D6B004302C295D297D2AF759F40020F233072C8
:100D7B0043207D20C2AF754303900175757E20C261
:100D8B0096C297306204D294A197D295D2AF759F39
:100D9B0041020F23C2AF754303900175757E20C2CC
:100DAB0092C293306204D294A1B7D295D2AF759F01
:100DBB0043020F23207D17C2AF754303900150C22E
:100DCB0096306202D294D2AF759F41020F23C2AF0D
:100DDB00754303900150C292306202D294D2AF7528
:100DEB009F43020F23207D11C2AF754304C293D2E0
:100DFB0097D2AF759F43020F23C2AF754304C297BF
:100E0B00D293D2AF759F41020F23307243207D20C6
:100E1B00C2AF754305900164757E08C294C29530CC
:100E2B006204D292C133D293D2AF759F40020F238B
:100E3B00C2AF754305900186757E80C294C2953012
:100E4B006204D296C153D297D2AF759F40020F2343
:100E5B00207D17C2AF754305900146C294306202E4
:100E6B00D292D2AF759F40020F23C2AF754305904C
:100E7B00015AC2943062EBD296D2AF759F40020FEB
:100E8B0023207D11C2AF754306C297D295D2AF75A1
:100E9B009F41020F23C2AF754306C293D295D2AFC7
:100EAB00759F43020F23307242207D20C2AF7543E2
:100EBB0001900186757E80C292C293306204D296F5
:100ECB00C1CFD297D2AF759F43020F23C2AF7543E9
:100EDB0001900164757E08C296C297306204D2926B
:100EEB00C1EFD293D2AF759F41E123207D16C2AFE4
:100EFB0075430190015AC292306202D296D2AF75FD
:100F0B009F43E123C2AF754301900146C296306205
:100F1B0002D292D2AF759F41C26622900144757E78
:100F2B0000C292C296C294C293C297C295C2622269
:100F3B00788076FF0876FF0876FF0876FF08760341
:100F4B0008760408760A0876030876010876017895
:100F5B008C76010876FF0876FF0876FF0876FF0887
:100F6B0076FF0876030876FF0876FF0876FF08768B
:100F7B00250876D00876FA0876FA0876040876FF04
:100F8B0008760108760008767A0876FF087601085D
:100F9B007601087600087603227887E6FFC272BFD7
:100FAB000302D2727888E6C394036008C27DE630F0
:100FBB00E102D27DC27E7889E630E102D27EC3EFB8
:100FCB0094026008758E01D273020FDC758E00C21D
:100FDB0073227880E6149000809378A4F67881E6EB
:100FEB00149000809378A5F67886E61490008D9384
:100FFB0078A6F6789CE67538FF75390CB402067541
:10100B0038A075390AB4030675388275390578A38B
:10101B00E61490009A93F569120F2622227896E631
:10102B00FA7897E6FB7888E6B40305C3EB940EFBDE
:10103B00307F047A007BFFC3EB9AFCC3948250028F
:10104B007C827575000575EC8575F0A4C3E5F0948D
:10105B007D40F222D27F11281205FB7A007B007CA7
:0E106B00101205F1E55F2AFA74003BFBDCF37E
:101079007C04C3EB13FBEA13FADCF7FEC27F1128E9
:1010890022E5EF20E6037520000520903FFFE520CB
:10109900146006901FFF1460009304600375EF123B
:1010A90053D9BF7581C043FF801205EC75EF024328
:1010B900B203E5B3240420E70DF521E5E320E006BA
:1010C9008521B343E301120F267580FF75A40075CE
:1010D900F13075D4DF75900375A5FC75F2FC75D5F3
:1010E9000175A60175E241C292C296C29412060028
:1010F900D293D297D2951205ECC293C297C295E4C6
:10110900F8F6D8FD756B01120F3B1215F278988627
:1011190076753001C2AF1206051206151205FB12CB
:10112900061C1205FB1206231205FB12170B1206E9
:1011390005120605120600C2AF78FA79FA3085075A
:10114900D9FBD8F7021C00120FA4120FDD112711C9
:101159002878988676120F2675B68075A900757D50
:101169000075885075891275C82475910475D84021
:1011790075A82275B80275E690759B80759D0075F6
:10118900D10E75BC5875BB0875BA1175E880120582
:10119900ECD2AF1208A553DACF207E0343DA203010
:1011A9007E0343DA1043DA01C2D8C271120605D2AE
:1011B900617B037A0CE55E70077A0CDB0302114050
:1011C9001205FB207003021140C270E55FC394024F
:1011D90040E1E52F541F856160F561B560D5DAD529
:1011E900C26153DACF207E0343DA20307E0343DA2B
:1011F90010C2D8C27178A2E67008D274E52F54E003
:10120900F52FC275752900120600307409C3E52946
:10121900940A4002D2751205F178023074027800FE
:10122900C3E55F9840F0C2AF120615120615120603
:1012390015D2AF120605754D007888E6B403026130
:10124900201205F1788CE6C394015003021320E5BE
:1012590030C394015003021320207435C3E55F9411
:10126900FF5003021320C2AF12062AD2AF120600A2
:10127900C3E55F940150EFC2AF1206151205F612CD
:101289000615D2AF120600C3E55F94FF40E90217C5
:10129900907F05D27F1128120600C2AFC27F1128A4
:1012A900AE5FC3E55F947FD2AF40761205ECC2AF63
:1012B90012062AD2AFDFDC115FC3EE94057897F6E8
:1012C9001206051216341217137F0AD27F1128123B
:1012D9000600C2AFC27F1128AE5FC3E55F947FD21B
:1012E900AF50E61205ECC2AF1206151205F612064A
:1012F90015D2AFDFD6115FEE24057896F6120605F2
:101309001216341217421206001128C3E55F94FF22
:1013190050024162021790C3E55F954D4003855F16
:101329004D12060078017988E7B403027805C3E510
:101339005F9840024142C2AF12062A12062A1206DB
:101349002AD2AF120605753000E4F531F5320531C0
:10135900E531F470390532789AE678191460127813
:101369003214600D787D14600878FA1460037532C0
:1013790000C3E53298401715327531B478998676ED
:10138900C2AF12062AD2AF789886761206001205E5
:10139900F6E52A700530740221407801207402783C
:1013A90006C3E55F9840A77888E6C39403600312F3
:1013B9000600E52A7003021140C2AF120F26E4F5B8
:1013C90022F523F524F525F526F56AD2AF7885E6C9
:1013D900C333F568E4F545F546F547F548F549F5AC
:1013E90073F52CF52DF53775730875BB101205ECDF
:1013F9001208A9E5E820ECFBA8BDA9BEE97001F82F
:1014090088741208AD75730875BB107887E6FE7687
:1014190002120FA47887EEF6C2AF7564FF12092590
:10142900852264852265852266D2AF7522017524DD
:101439000175250175260185636C756D0175B69079
:1014490075A903757D017888E6B40307C27D3076F6
:1014590002D27DD268D269753300120E8C120EB198
:0F14690012094512094C12094512094C12094586
:10147800021488C2AF120FA4D2AF75730075BB08EF
:10148800120BDE1206F5120D0A120D5412094C1237
:101498000BCD306D031206F620670312084830673B
:1014A8000312088F120D0A120D7912094C120BDE65
:1014B800306D03120732120D0A120DF012094C1288
:1014C8000BCD306D03120790120D0A120E1512097A
:1014D8004C120BDE306D031207ED120D0A120E8C42
:1014E80012094C1208A9120BCD120D0A120EB112D4
:1014F80008AD12094C306932206B2F856764856707
:101508006585636C756D0179187A0CC3E53399406C
:101518000CC269D26A8A357564FF021532C3E55F69
:10152800940140030214880215AF306A1B206B181F
:10153800E535147004C26A817BF535C3E55F940113
:1015480040030214880215AF753600C3E56278823D
:10155800985054307404E52A604D7888E6B403172F
:10156800207D05207607A17F307602A17F206B07BA
:10157800D26B85676481C778F0306B0585676478BE
:1015880020C3E5419850028188306B1BC26BC27D35
:10159800307602D27DD26A753512856764818805F6
:1015A80036E55F6002A1B2753600C2AF120F267829
:1015B80087E6FE7602120FA47887EEF6E4F522F5A8
:1015C80023F524F525F526F568C26875B68075A952
:1015D80000757D00D2AF1205EC120F26307409C3D6
:1015E800E5369405400221406152901A0D78201288
:1015F8001676E520B45A0CA3121676E520B4A50396
:10160800021614120F3B121634021633901A03787E
:10161800807B0A121676A308DBF9901A0F788C7B68
:1016280018121676A308DBF9901A2722C2AF1216F1
:10163800B512168F901A00740E12167BA37404123A
:10164800167BA3741412167B901A0378807B0A12F7
:10165800167AA308DBF9901A0F788C7B1812167A81
:10166800A308DBF91216C81216A6901A2722E493CB
:10167800F622E6438F01538FFD75EF0275B7A57506
:10168800B7F1F0538FFE22438F02438F0175EF02AB
:1016980075B7A575B7F1901A0DF0538FFC22901A03
:1016A8000D745AD17B901A0E74A5D17B227A3079A9
:1016B800D07820901A40D176E520F709A3DAF722EE
:1016C8007A3079D0901A40E7D17B09A3DAF922ABB6
:1016D80077A878BB01027984BB02027985BB030233
:1016E8007986BB04027992BB05027987BB06027929
:1016F800A3BB0702799CBB08027988BB09027989D8
:10170800E8F7227C05120605DCFB22C2AF1206159B
:1017180012061C12062312062A1205F612061512C4
:10172800061C12062312062A1205F61206151206C0
:101738001C12062312062AD2AF22C2AF12062A12A0
:10174800062312061C1206151205F612062A1206A0
:101758002312061C1206151205F612062A12062373
:1017680012061C120615D2AF22AE77AF78C2AF129E
:1017780006151206151206151205F6DEF212062ACD
:101788001205F6DFF8D2AF22F113F10BF10B7577E2
:1017980001757801757900F1717C05AD5F12060558
:1017A800C3ED955F70F5C3E55F9401400AC3E55F3B
:1017B80094FF40320217CCD1D7D134F113C2AF75A0
:1017C800EF12F10BDCD50579C3E57994035002805B
:1017D800C6F10B0578E5771490009F93F808C3E5E8
:1017E8007898500280AEF10BF10B0577C3E577943A
:1017F8000A5002809C120F3B121634C2AF75EF12CA
:0318080012170BA9
:0319FD0002108A4B
:101A00000E0414FFFFFFFF03040A0301015AA5019E
:101A1000FFFFFFFFFF03FFFFFF25D0FAFA04FF01DE
:081A2000007AFF01010003FF41
:101A400023475F556C74726132304123202020207F
:101A500023424C48454C492346333930232020202B
:101A60002020202020202020202020202020202076
:101C0000C2AFC2D353D9BF7581C043B20343FF8073
:101C1000752438752503B1C975EF0275E24043F1AB
:101C20002053A4DF75D400D2857DFA780379E67C51
:101C300010752200752300901DD67B0675249875BB
:101C400025013085028142208508D8FBD9F9DCF7CF
:101C500081B4308508D8FBD9F9DCF781B4B189E4C7
:101C600093A3C39A6004DDC381B4DBDBB17B600264
:101C7000812B7B08E493FAA3B15CDBF87A30B15C8A
:101C8000752200752300B17BEAFCEBFDC3ED94FEE9
:101C9000400EB17B8A278B28ED30E0048A828B834B
:101CA000B17B7AC270D8C3ED94FE601350CEBD00F4
:101CB00025EC60097520007521FF0200008100A855
:101CC00027A9280809D804D90281D3B17FEA89AAB3
:101CD000F281C50D81A0C3ED94035049EDA2E092BD
:101CE000007AC5C3E5829400E583941C50902000DF
:101CF00010438F02438F0175B7A575B7F1F030001F
:101D00001FA827A9280809438F01538FFDD804D99C
:101D100002A12089AAE275B7A575B7F1F0A3A10DBC
:101D2000538FFC817C7AC1BD030CE493A3FAB140CC
:101D3000DCF8B138817C817EAA22AB23B15CEBFA5E
:101D4000EA6222752608C3E52313F523E52213F57D
:101D50002250066323A0632201D526EAB1C9B1C986
:101D600075260AEAF4200102D285300102C285B14B
:101D7000C9C3134002C201D526EB22B17FEAFB2082
:101D80008502A17F308502A184752608AE24AF2587
:101D9000C3EF13FFEE13FEB1CDB1C9C3EA13308513
:101DA000024480FA30E703632201C3E52313F523DD
:101DB000E52213F52250066323A0632201D526D91C
:101DC000E52265236523F52222AE24AF250E0FDE22
:101DD000FEDFFCD20122424C48656C693437316326
:041DE000F390060175
:00000001FF
